:020000020000FC
:100000000C949C020C9447060C9447060C944706EB
:100010000C9447060C9447060C9410060C94470663
:100020000C9447060C9441060C9447060C94470622
:100030000C9447060C9447060C9423060C94470630
:100040000C9447060C9447060C9447060C944706FC
:100050000C94470608958AD1EEF7E8940CECFBD196
:1000600004E4F9D1B9D3F4D263D3B0D10F3FD1F7BF
:100070007DD1B6F5E8940CECEED10EEBECD1A6D127
:1000800000936200A3D10093630000916300007F9E
:10009000003021F001E00093660003C000270093C8
:1000A0006600009162000F7000936400009162008E
:1000B000007F109163001770010F02950093650097
:1000C00000916600003061F00091650000950F77A7
:1000D000009365000091640010E1101B1093640010
:1000E00001D00895009164000150A0F00250B0F0DA
:1000F0000250C0F00250D0F00250E0F00250F0F098
:10010000025000F1025010F1015020F119E010935B
:100110006400089510E010936400089511E01093B6
:100120006400089512E010936400089513E01093A2
:100130006400089514E010936400089515E010938E
:100140006400089516E010936400089517E010937A
:100150006400089518E0109364000895089516D17E
:10016000EEF7E8940CEC8ED104E48CD135D370D248
:10017000DFD243D10F3FD1F709D1B6F5E8940CECAB
:1001800081D10EEB7FD139D10093670036D1009336
:10019000680000916800007F003021F001E00093CA
:1001A0006B0003C0002700936B00009167000F7085
:1001B0000093690000916700007F1091680017703C
:1001C000010F029500936A0000916B00003061F00E
:1001D00000916A0000950F7700936A000091690012
:1001E00010E1101B1093690001D00895009169007F
:1001F0000150A0F00250B0F00250C0F00250D0F018
:100200000250E0F00250F0F0025000F1025010F104
:10021000015020F119E010936900089510E0109347
:100220006900089511E010936900089512E0109399
:100230006900089513E010936900089514E0109385
:100240006900089515E010936900089516E0109371
:100250006900089517E010936900089518E010935D
:10026000690008950895A2D0EEF7E8940CEC21D12E
:1002700004E41FD1B1D2ECD15BD2D6D00F3FD1F77D
:1002800095D0B6F5E8940CEC14D10EEB12D1CCD08D
:1002900000936C00C9D000936D0000916D00007F49
:1002A000003021F001E00093700003C000270093AC
:1002B000700000916C000F7000936E0000916C0054
:1002C000007F10916D001770010F029500936F0071
:1002D00000917000003061F000916F0000950F7781
:1002E00000936F0000916E0010E1101B10936E00E0
:1002F00001D0089500916E000150A0F00250B0F0BE
:100300000250C0F00250D0F00250E0F00250F0F085
:10031000025000F1025010F1015020F119E0109349
:100320006E00089510E010936E00089511E0109390
:100330006E00089512E010936E00089513E010937C
:100340006E00089514E010936E00089515E0109368
:100350006E00089516E010936E00089517E0109354
:100360006E00089518E010936E000895B89AC09832
:1003700033D232D231D2C09AB8982CE3B1D068943B
:10038000B099E89429D228D227D20895B99AC19871
:1003900023D222D221D2C19AB9982CE3A1D0689459
:1003A000B199E89419D218D217D20895BA9AC2987E
:1003B00013D212D211D2C29AB9982CE391D0689478
:1003C000B299E89409D208D207D20895F89418E0B7
:1003D0000027B89AC09822E083D0C09AB898889431
:1003E000B099089407952BE37BD0B89AC09A81D036
:1003F00080D01A9571F778940895F89418E0002742
:10040000B99AC19822E06CD0C19AB9988894B199F0
:10041000089407952BE364D0B99AC19A6AD069D041
:100420001A9571F778940895F89418E00027BA9A0D
:10043000C29822E055D0C29ABA988894B29908948A
:1004400007952BE34DD0BA9AC29A53D052D01A9541
:1004500071F778940895F89418E0B89AC09822E05B
:100460003FD08894079518F02BE33AD003C0C09A88
:100470002BE336D0B89AC09A3CD03BD01A9569F796
:1004800078940895F89418E0B99AC19822E028D099
:100490008894079518F02BE323D003C0C19A2BE36F
:1004A0001FD0B99AC19A25D024D01A9569F77894AB
:1004B0000895F89418E0BA9AC29822E011D088946E
:1004C000079518F02BE30CD003C0C29A2BE308D099
:1004D000BA9AC29A0ED00DD01A9569F778940895F9
:1004E0002A952A9500000000000000000000C9F7CE
:1004F0000895000008952F936FD12F912A95D9F771
:100500000895E199FECF1EBBF898E09A0DB30895C7
:100510000000E199FDCFF8941EBBF8980DBBE29A5C
:10052000E19A789408951AE0ECDF009374001BE0E0
:10053000E8DF00937D00089504E00EBF0FE50DBFD6
:100540000DE30ABB03E00BBB08EF07BB07E008BBEA
:100550000FEF01BB04BB0CE005BB002702BB0093FF
:1005600081000093800000937E0000936000009360
:10057000610000937F00009373000CE0009375000E
:100580000093760000937700009378000093790041
:1005900000937A0000937B0000937C00222403E008
:1005A00003BF04E00EBD1AE702E11BBD0ABD01E175
:1005B00009BF002702BF0DBD0CBD0EE806B906E05D
:1005C00007B978940DD082D1AEDFB2D005D140D03A
:1005D00042DDAED0C4DDACD046DEAAD001D0F5CF2E
:1005E00000917400003039F0013041F0023049F0E0
:1005F000AC9AAD9A0895AC98AD980895AD9AAC9820
:100600000895AD98AC9A0895009161000B3321F0E4
:10061000039500936100089510916000133671F006
:1006200013951093600000270093610008950091D6
:100630007D00033061F400270093800000270093C1
:1006400060000093610074D0C7D0C89BFDCF0895AF
:1006500002E0202EC89B03C0C99B0BC00895BCD0EC
:10066000022D003021F0C89BFACF3BD00895DFDF88
:100670000895B2D0C89B04C0C99BFBCF0AD008958F
:10068000ABD0C89BFDCF1DD0ABDF01E00093810054
:10069000089500918100013081F000917D000330C8
:1006A00031F0039500937D001BE032DF08950027B1
:1006B00000937D001BE02CDF08950027009381004C
:1006C000089500917400033031F003950093740095
:1006D0001AE01EDF08950027009374001AE018DF67
:1006E000089500917D00033059F40091800001309D
:1006F00021F001E00093800008950027009380001E
:10070000089500917E00003491F4009171001091E1
:10071000720026E0169507952A95E1F7009373007D
:10072000002700937E0000937100009372000895EB
:10073000009164001091650020916600FCD1009347
:100740007500109376002093770030937800009125
:100750007D00003039F00130A9F0023091F1033012
:1007600009F108950091690010916A0020916B00D1
:10077000E2D10093790010937A0020937B003093AC
:100780007C00089500916E0010916F002091700020
:10079000D2D10093790010937A0020937B0030939C
:1007A0007C00089510916100CBD1109379002093C3
:1007B0007A0010916000C4D110937B0020937C00DC
:1007C00008959FDFF1D10093790010937A00209370
:1007D0007B0030937C000895109178005BD012BBB1
:1007E000F894A89A68D078941091770053D0A8987C
:1007F00012BBF894C79A5FD07894109176004AD0D3
:10080000C79812BBF894C69A00917D000A3009F08F
:10081000959851D07894109175003CD0C69812BB31
:10082000F894C59A48D0789410917C0033D0C5983C
:1008300012BBF894A99A3FD0789410917B002AD0EB
:10084000A99812BB00917D00023019F0033009F025
:1008500001C09598F894AB9A2ED0789410917A00B4
:1008600019D0AB9812BB00917D00003019F0013017
:1008700009F001C09598F894C39A1DD0789410910E
:10088000790008D0C39812BBF894C49A14D0C498C5
:1008900078940895E4EAF8E020E0E10FF21FC895AB
:1008A000102D089521F92AA8F0A424E920A0267E7D
:1008B000FFFE70373DFF1F932F9312E32AE01A9536
:1008C000F1F72A95E1F72F911F9108950AE000931F
:1008D0007D000DE00093750000937C0027D10DE0B2
:1008E000009375000093760000937B0000937C00DA
:1008F0001DD10DE000937500009376000093770002
:1009000000937C0000937B0000937A000FD10DE0F0
:1009100000937500009376000093770000937800B1
:1009200000937C0000937B0000937A000093790091
:10093000FDD00DE0009375000093760000937700E2
:100940000093780000937C0000937B0000937A0072
:1009500000937900EBD00DE00093780000937700CE
:100960000093760000937B0000937A000093790057
:100970000CE00093750000937C00D8D00DE000934C
:1009800078000093770000937A00009379000CE0E0
:10099000009375000093760000937C0000937B0029
:1009A000C5D00DE000937800009379000CE000932F
:1009B0007500009376000093770000937C0000930D
:1009C0007B0000937A00B2D00CE000937500009396
:1009D00076000093770000937C0000937B000093E7
:1009E0007A000093780000937900A0D00EE0009385
:1009F00079009CD00EE000937A000AE00093790021
:100A000095D00EE000937B000AE000937A000FE09F
:100A1000009379008BD00EE000937C000AE00093F5
:100A20007B000FE000937A000FE0009379007ED006
:100A30000EE0009375000AE000937C000FE0009345
:100A40007B000FE000937A0000E0009379006ED005
:100A50000EE0009376000AE0009375000FE000932B
:100A60007C000FE000937B0000E000937A000CE034
:100A7000009379005BD00EE0009377000AE00093CA
:100A800076000FE0009375000FE000937C0000E01B
:100A900000937B000CE000937A000093790046D02D
:100AA0000EE0009378000AE0009377000FE00093D7
:100AB00076000FE00093750000E000937C000CE0EE
:100AC00000937B0033D00AE0009378000FE000939E
:100AD00077000FE00093760000E0009375000CE0D3
:100AE00000937C0023D00FE0009378000FE0009388
:100AF000770000E0009376000CE00093750016D0BC
:100B00000FE00093780000E0009377000CE0009382
:100B100076000CD000E0009378000CE000937700A2
:100B200005D00CE00093770001D00895A7ED54DEC6
:100B3000A395E9F70895203011F03DE001C03CE0B5
:100B40001A50B8F01A50E8F01A50E8F01A50E8F0CD
:100B50001A50E8F01A50E8F01A50E8F01A50E8F08D
:100B60001A50E8F01A50E8F02AE01BE00BE03CE0F5
:100B7000089520917D00233011F02CE013C022272E
:100B800011C021E00FC022E00DC023E00BC024E023
:100B900009C025E007C026E005C027E003C028E023
:100BA00001C029E0165F089500917300085C30F4DD
:100BB0000853045640F0045631E006C03CE02AE0F9
:100BC0001BE00BE008953CE00C590A5098F00A50E5
:100BD00098F00A5098F00A5098F00A5098F00A508D
:100BE00098F00A5098F00A5098F00A5098F00A507D
:100BF00029E012C020E010C021E00EC022E00CC0AD
:100C000023E00AC024E008C025E006C026E004C0B6
:100C100027E002C028E000C0065F102F00E1089521
:100C20000F931F939FB700270DBD0CBD022D003001
:100C300009F02A9400918000013009F4E5DC9FBF9F
:100C40001F910F9118950F931F932F933F939FB769
:100C500000917E00003479F0039500937E0014B17A
:100C600005B12091720030917100310F201F309337
:100C70007100209372009FBF3F912F911F910F91A0
:100C800018950F931F93369A1F910F9118951895E9
:00000001FF
